:1000000083168601831246207C200E306020A020BB
:10001000A60126082320003E031912286E20A020E6
:10002000A60A0928A60AC0306020A020260823209E
:10003000003E03191F286E20A020A60A16280130B2
:100040006020A020082882075334503445344334BC
:100050005434523455344D34CE34B034D134CD349C
:10006000DF34B034BC34DE34003430343134323434
:100070003334343435343634373438343934413425
:100080004234433444344534463400349820982074
:100090003030672098203030672091203030672042
:1000A0009120203067207C20283060207C20083080
:1000B00060207C20013060207C2006306020080019
:1000C000A500F0396720250EF0396720080086006A
:1000D000861006110614000006100800A500F0396D
:1000E0007520250EF039752008008600861006154B
:1000F00006140000061008008316F03086008312F4
:1001000006118614061406080610A5000614060833
:100110000610A51B7C2886108316003086008312EB
:100120000800A530A00000000000A00B95280800E2
:100130006330A100000000009120A10B9C28080062
:100140006330A2006230A3000330A40000009820B6
:10015000A20BA7289120A30BAA28A40BAD28080066
:00000001FF
